:100000000C9435000C945D000C945D000C945D0024
:100010000C945D000C945D000C945D000C945D00EC
:100020000C945D000C945D000C945D000C945D00DC
:100030000C945D000C945D000C945D000C945D00CC
:100040000C945D000C945D000C9428060C946306DF
:100050000C945D000C945D000C945D000C945D00AC
:100060000C945D000C945D00CF0711241FBECFEFF0
:10007000D4E0DEBFCDBF11E0A0E0B1E0E8E2F1E105
:1000800002C005900D92AC31B107D9F711E0ACE197
:10009000B1E001C01D92A63DB107E1F710E0CAE64C
:1000A000D0E004C02297FE010E948E08C836D10716
:1000B000C9F70E940F060C9492080C940000DC0112
:1000C000FC01672F71917723E1F7329704C07C918F
:1000D0006D9370836291AE17BF07C8F30895282F00
:1000E00080931D0188309CF484E290E0909322017B
:1000F0008093210185E290E0909325018093240173
:1001000083E290E0909328018093270133C08031EF
:10011000C4F487E290E0909322018093210188E269
:1001200090E0909325018093240186E290E09093E3
:10013000280180932701332727FD30952850304030
:1001400019C0883104F58AE290E0909322018093EF
:1001500021018BE290E0909325018093240189E2B4
:1001600090E09093280180932701332727FD309555
:100170002051304081E090E002C0880F991F2A95FD
:10018000E2F780932301E0912401F0912501808121
:1001900090912301892B8083E0912101F09122012C
:1001A00080819095892380830895EF92FF920F9329
:1001B0001F938430910518F484E090E005C08938DD
:1001C000910510F088E890E0A0E0B0E07C018D019E
:1001D00034E0EE0CFF1C001F111F3A95D1F722EFFF
:1001E000E216F1040105110544F482E090E09093D9
:1001F000200180931F0181E018C0880F991FAA1F5A
:10020000BB1F823F9105A105B10544F480E190E058
:100210009093200180931F0182E007C080E490E06A
:100220009093200180931F0183E080931C01209113
:100230001F013091200140E050E0C801B7010E9449
:10024000710820931E0130E03595279520932601F3
:100250001F910F91FF90EF900895CF92DF92EF9250
:10026000FF920F931F93DF93CF9300D000D0CDB7B1
:10027000DEB78C01242F49835A836B837C836E0104
:100280000894C11CD11C4BE2E42E41E0F42EC701BE
:10029000B801422F0E941C060F5F1F4FC701B80113
:1002A000F60141810E941C060F5F1F4FC701B80174
:1002B000F60142810E941C060F5F1F4FC701B80163
:1002C000F60143810E941C060F900F900F900F9033
:1002D000CF91DF911F910F91FF90EF90DF90CF9022
:1002E0000895CF92DF92EF92FF920F931F93CF93D7
:1002F000DF936B017C01EA0100E0C701B6012AE04F
:1003000030E040E050E00E944F08162FC701B601D0
:100310002AE030E040E050E00E944F08C901DA01D5
:100320006C017D01FE01E00FF11D105D10830F5F78
:10033000C114D104E104F10401F7CE01800F911D35
:100340008C01FC011082CE010E945F00C801DF9188
:10035000CF911F910F91FF90EF90DF90CF90089574
:10036000CF93DF93EC016115710519F420E030E0C3
:100370000FC0DB010D900020E9F71197A61BB70B0A
:10038000E881F9810280F381E02DAD0109959C019E
:10039000C901DF91CF9108952F923F924F925F92C2
:1003A0006F927F928F929F92AF92BF92CF92DF9285
:1003B000EF92FF920F931F93DF93CF93CDB7DEB7EA
:1003C000C053D1400FB6F894DEBF0FBECDBFF89436
:1003D00015BC14BC10928100109280001092B100E4
:1003E0001092B0008BE291E060E070E00E94150690
:1003F000813681F48BE291E061E070E00E941506A5
:10040000853741F48BE291E062E070E00E941506CE
:100410008C3691F18BE291E060E070E041E60E9461
:100420001C068BE291E061E070E045E70E941C064B
:100430008BE291E062E070E04CE60E941C068BE2E9
:1004400091E063E070E041E00E941C068BE291E0E5
:1004500064E070E042E10E941C068BE291E065E0FE
:1004600070E040E20E941C0686E090E040E05BE421
:1004700060E070E00E942D018BE291E064E070E0AA
:100480000E9415060E946F008BE291E065E070E02B
:100490000E94150690E00E94D5008E010F5F1F4F4D
:1004A0008BE291E066E070E00E94150689838BE2A2
:1004B00091E067E070E00E941506D80111968C93D8
:1004C0008BE291E068E070E00E941506F8018283FB
:1004D0008BE291E069E070E00E941506D801139666
:1004E0008C9349815A816B817C81409307015093A1
:1004F00008016093090170930A0184EB91E00E9466
:100500009E06789480911C018093B100FE0135967F
:100510008CE291E0DF019C011D9221503040E1F717
:100520008FEF8D838E838FE78F83EE2482E0C82E3A
:100530005F0108E0602E712C6C0E7D1E10E5312EDF
:10054000B9E04B2E512C4C0E5D1EAAE3DA2EF2E4DC
:100550002F2EECE08E2E912C8C0E9D1E01C0EF2CC8
:1005600084EB91E00E942507892B09F45EC284EB9D
:1005700091E00E94560735E03093B100C3BC03B44C
:1005800001FCFDCF88871092B20004E010E084EBFC
:1005900091E00E942507892B61F084EB91E00E9495
:1005A0005607F501E00FF11F80830F5F1F4F109278
:1005B000B2008091B200803D50F380911C01809385
:1005C000B1008885843209F08BC189858D3409F0AA
:1005D00087C18A858C3309F083C10A0D1B1DD801A0
:1005E0001C928B858035C9F1813520F4823409F065
:1005F000D6C007C0823509F45CC0873509F0CFC08A
:100600009BC0F40120E030E040E050E01FC0DA0180
:10061000C901880F991FAA1FBB1F03E0220F331FB8
:10062000441F551F0A95D1F7280F391F4A1F5B1F1A
:10063000862F992787FD9095C097AA2797FDA095AB
:10064000BA2F280F391F4A1F5B1F3196608166231E
:10065000F1F6C9010E94D500A2C0F40120E030E00B
:1006600040E050E01FC0DA01C901880F991FAA1F9E
:10067000BB1F73E0220F331F441F551F7A95D1F71C
:10068000280F391F4A1F5B1F862F992787FD9095DA
:10069000C097AA2797FDA095BA2F280F391F4A1F88
:1006A0005B1F319660816623F1F6822F0E946F00F6
:1006B00076C0F40120E030E040E050E01FC0DA01F5
:1006C000C901880F991FAA1FBB1F13E0220F331FF8
:1006D000441F551F1A95D1F7280F391F4A1F5B1F5A
:1006E000862F992787FD9095C097AA2797FDA095FB
:1006F000BA2F280F391F4A1F5B1F3196608166236E
:10070000F1F62093070130930801409309015093BB
:100710000A01205835424040504060F480E895E29C
:10072000A0E0B0E08093070190930801A093090135
:10073000B0930A0111E034C08BE291E064E070E014
:1007400040911D010E941C0680911E0190E02091A5
:100750001F0130912001829FA001839F500D929F25
:10076000500D1124B4E056954795BA95E1F78BE208
:1007700091E065E070E00E941C06409107015091F5
:1007800008016091090170910A0186E090E00E94E1
:100790002D0184EB91E060E071E00E94B00110E077
:1007A000F301308260911D01772767FD7095872FD7
:1007B000972FA2010E947101FC01D0822182329602
:1007C00080911E0190E020911F0130912001829FB5
:1007D000B001839F700D929F700D1124A4E0769557
:1007E0006795AA95E1F780E090E0AF010E94710162
:1007F000FC01D08222E5218332966091070170913D
:1008000008018091090190910A01AF010E947101D4
:10081000DC01FC01D19211963C92119739E43183AD
:100820008EE4828393E59383D48216962C92169756
:10083000179660E070E080E090E0AD010E947101E9
:10084000DC01FC01D19283E411968C93319668E02F
:1008500070E080E090E0AF010E947101DC01FC01DA
:10086000D19284E411968C93319660E170E080E03F
:1008700090E0AF010E947101FC01D082118284EBF3
:1008800091E0B3010E94B00184EB91E06AE00E9424
:100890008F07112309F464CE84EB91E00E947F0757
:1008A000A5E0A093B1001092B2008091B200803D0B
:1008B000E0F31092B2008091B200803DE0F38091AD
:1008C0001C018093B1004091070150910801609193
:1008D000090170910A0184EB91E00E949E0640CECE
:1008E000E0912101F0912201808190912301892BD7
:1008F0008083C3BC03B401FCFDCF3091260140E0EE
:1009000050E0F501E40FF51F8081A1E060E070E0A8
:10091000E82EFF248A2F90E08E219F212091230131
:10092000E0912401F0912501892BF1F08081822B47
:1009300080831092B20090911E018091B2008917BD
:10094000E0F3E0912401F091250190818091230151
:100950008095982390831092B20090911E0180910F
:10096000B2008917E0F338C08081822B8083109217
:10097000B2008091B2008317E0F3E0912401F0917E
:100980002501908180912301809598239083109276
:10099000B2008091B2008317E0F3E0912401F0915E
:1009A0002501808190912301892B80831092B200D0
:1009B0008091B2008317E0F3E0912401F0912501CA
:1009C0009081809123018095982390831092B200AA
:1009D0008091B2008317E0F3AA0F6F5F7F4F6830FA
:1009E000710509F097CF4F5F5F4F401751070CF427
:1009F00088CFE0912401F09125018081909123011D
:100A0000892B80831092B2008091B2008317E0F3AB
:100A1000E0912101F0912201908180912301809544
:100A200098239083EE24E3949BCDE0912701F091ED
:100A30002801F08080912301F822EE2009F08FCD6B
:100A4000FF2009F48CCDC3BC03B401FCFDCF40E012
:100A5000282F332727FD30951092B20005C08091D2
:100A6000B2008B3F08F07BCD808190E082239323FE
:100A7000892BA9F705C08091B2008B3F08F06FCD9C
:100A8000808190E082239323892BA9F34F5F493023
:100A900019F71092B20005C08091B2008B3F08F0A8
:100AA0005ECD808190E082239323892BA9F705C036
:100AB0008091B2008B3F08F052CD808190E082237C
:100AC0009323892BA9F38091B20080932A0190E0AF
:100AD0009C01359527959595879595958795082F30
:100AE000020F00932901A0912701B0912801809164
:100AF0002301282F332727FD30951092B20005C01F
:100B00008091B2008B3F08F02ACD8C9190E0822337
:100B10009323892BA9F705C08091B2008B3F08F081
:100B20001ECD8C9190E082239323892BA9F3809191
:100B3000B200081710F31092B20005C08091B20005
:100B40008B3F08F00CCD8C9190E082239323892B6E
:100B5000A9F705C08091B2008B3F08F000CD8C91C1
:100B600090E082239323892BA9F343E050E010E027
:100B700060E070E01092B20005C08091B2008B3F3F
:100B800008F045C08C9190E082239323892BA9F72C
:100B900004C08091B2008B3FD0F58C9190E082230D
:100BA0009323892BB1F38091B200081710F481E0F0
:100BB00019C01092B20004C08091B2008B3F38F58A
:100BC0008C9190E082239323892BB1F704C080910C
:100BD000B2008B3FE0F48C9190E082239323892B29
:100BE000B1F380E090E0062E02C0880F991F0A94AE
:100BF000E2F7182B6F5F7F4F6830710509F0BACFAD
:100C0000F501E40FF51F10834F5F5F4FB0CF4350E6
:100C1000504084EB91E0B3010E942508A0CC80E015
:100C20000E94CC0180E090E00895F999FECF72BD5A
:100C300061BDF89A80B50895F999FECF1FBA72BDCB
:100C400061BD40BD0FB6F894FA9AF99A0FBE0895A7
:100C50001F920F920FB60F9211242F933F934F9331
:100C60008F939F93EF93FF938091C00082FD1DC0EF
:100C70004091C60020916C0130916D012F5F3F4F74
:100C80002F73307080916E0190916F012817390792
:100C900071F0E0916C01F0916D01E45DFE4F4083D5
:100CA00030936D0120936C0102C08091C600FF91CA
:100CB000EF919F918F914F913F912F910F900FBE88
:100CC0000F901F9018951F920F920FB60F9211243C
:100CD0002F933F938F939F93EF93FF932091B001B6
:100CE0003091B1018091B2019091B3012817390779
:100CF00031F48091C1008F7D8093C10014C0E091D8
:100D0000B201F091B301E059FE4F20818091B20110
:100D10009091B30101968F7390709093B30180937B
:100D2000B2012093C600FF91EF919F918F913F9167
:100D30002F910F900FBE0F901F901895AF92BF92FA
:100D4000DF92EF92FF920F931F93CF93DF93EC010B
:100D50007A018B01DD24403081EE580780E068077E
:100D600080E0780711F0DD24D39491E0A92EB12C16
:100D7000EC89FD89DD2069F0C50108A002C0880F5B
:100D8000991F0A94E2F7808360E079E08DE390E0B8
:100D900005C0108260E874E88EE190E0A801970138
:100DA0000E944F0821503040404050405695479592
:100DB0003795279580E12030380720F0DD2011F0AD
:100DC000DD24D6CFE889F9893083EA89FB8920833D
:100DD00019A2EE89FF89408121E030E0C9010C8C25
:100DE00002C0880F991F0A94E2F7482B4083EE89CE
:100DF000FF894081C9010D8C02C0880F991F0A9498
:100E0000E2F7482B4083EE89FF894081C9010E8CAF
:100E100002C0880F991F0A94E2F7482B4083EE899D
:100E2000FF8980810F8C02C0220F331F0A94E2F7E2
:100E3000209528232083DF91CF911F910F91FF9060
:100E4000EF90DF90BF90AF900895DC011C96ED917C
:100E5000FC911D97E05CFF4F219131918081918140
:100E6000281B390B2F733070C9010895DC011C96C3
:100E7000ED91FC911D97E05CFF4F20813181E054A2
:100E8000F040DF01AE5BBF4F8D919C911197281709
:100E9000390719F42FEF3FEF07C08D919C91E80FB0
:100EA000F91F8081282F30E0C9010895DC011C96CC
:100EB000ED91FC911D97E05CFF4F20813181E05462
:100EC000F040DF01AE5BBF4F8D919C9111972817C9
:100ED000390719F42FEF3FEF10C08D919C911197B6
:100EE000E80FF91F20818D919C91119701968F73C6
:100EF000907011969C938E9330E0C9010895DC01A7
:100F000091968C919197882339F05496ED91FC91AC
:100F10005597808186FFF9CF91961C920895CF93C3
:100F2000DF93EC01EE85FF85E05CFF4F208131818E
:100F3000E054F0402F5F3F4F2F733070DF01AE5B06
:100F4000BF4F8D919C91119728173907D1F3E05C21
:100F5000FF4F80819181E054F040E80FF91F6083DA
:100F6000EE85FF85E05CFF4F31832083EE89FF89AA
:100F7000208181E090E00F8C02C0880F991F0A94B5
:100F8000E2F7282B208381E089A3EC89FD89808109
:100F90008064808381E090E0DF91CF91089510928A
:100FA000B7011092B60188EE93E0A0E0B0E0809324
:100FB000B8019093B901A093BA01B093BB018FE03F
:100FC00091E09093B5018093B4018CE291E090930D
:100FD000C1018093C00180E791E09093C3018093A9
:100FE000C20185EC90E09093C5018093C40184EC2C
:100FF00090E09093C7018093C60180EC90E09093BD
:10100000C9018093C80181EC90E09093CB0180935B
:10101000CA0182EC90E09093CD018093CC0186ECE4
:1010200090E09093CF018093CE0184E08093D00133
:1010300083E08093D10187E08093D20185E08093A3
:10104000D30181E08093D4010895CF92DF92EF9293
:10105000FF920F931F93CF93DF937C016B018A0163
:10106000C0E0D0E00FC0D6016D916D01D701ED91C8
:10107000FC910190F081E02DC7010995C80FD91F9F
:10108000015010400115110571F7CE01DF91CF918C
:101090001F910F91FF90EF90DF90CF900895A1E204
:1010A0001A2EAA1BBB1BFD010DC0AA1FBB1FEE1FE2
:1010B000FF1FA217B307E407F50720F0A21BB30B2D
:1010C000E40BF50B661F771F881F991F1A9469F7A9
:1010D00060957095809590959B01AC01BD01CF0105
:1010E000089597FB092E05260ED057FD04D0D7DFB3
:1010F0000AD0001C38F450954095309521953F4F0B
:101100004F4F5F4F0895F6F79095809570956195D4
:101110007F4F8F4F9F4F0895EE0FFF1F0590F49163
:08112000E02D0994F894FFCFC3
:1011280073617665643A00004B0000000000008F90
:0C1138000725082507560736077F07002B
:00000001FF
